:100000008A01162832284D285A28622869289F28F4
:10001000B1288529B129B529E129E529112A152A0F
:10002000362A612A662A6B2A702A842A83160313C9
:100030009B01C03081000220032011203A30FD00D6
:10004000042012203A30FD000420132083120313F1
:10005000A2010130A30007201020C830F7000F20B4
:100060001C2831288316831603130608C03986001E
:1000700083120230F7000F203330FE0005203230AB
:10008000FE0005202C30FE0005200630FE00052075
:100090000C30FE000520032008000130FE00052082
:1000A0000130F7000F200230FE0005200130F7007C
:1000B0000F2008007D08FF00103083120313A000FA
:1000C000062008007E08FF0083120313A00106200B
:1000D00008007F08F000F00CF00CF00C700C0F39E9
:1000E0000F39831203132004A1000608C03921042C
:1000F000A10086000130F7000F208312031386163B
:100100000130F7000F208312031386127F080F3986
:100110002004A1000608C0392104A1008600013096
:10012000F7000F208312031386160130F7000F200B
:100130008312031386120130F7000F200800831288
:100140000313A308031DA7288030A300A928C030EB
:10015000A300F001230822070318F00AFE0005207F
:1001600008000830F000F1010830F200F3018312BA
:1001700003132408F4000310F41B0314F30D64307C
:10018000F3020318C528F3070310F40DF20BBB2884
:100190007408F2000310F21B0314F10D0A30F1028F
:1001A0000318D428F1070310F20DF00BCA287108C8
:1001B000FF39003C03190B29F0013030F100083001
:1001C000F200F3010830F400F5012408F6000310F2
:1001D000F61B0314F50D6430F5020318F128F5073A
:1001E0000310F60DF40BE7287608F4000310F41B57
:1001F0000314F30D0A30F30203180029F307031068
:10020000F40DF20BF628730871070318F00AFF00CB
:100210001030A00006200830F000F1010830F20094
:10022000F301831203132408F4000310F41B0314D6
:10023000F30D0A30F30203181F29F3070310F40D1E
:10024000F20B15297408F2000310F21B0314F10DD0
:100250000A30F10203182E29F1070310F20DF00BFA
:1002600024297108FF39003C03196529F001303059
:10027000F1000830F200F3010830F400F501240821
:10028000F6000310F61B0314F50D0A30F5020318EF
:100290004B29F5070310F60DF40B41297608F400FD
:1002A0000310F41B0314F30D0A30F30203185A2948
:1002B000F3070310F40DF20B5029730871070318AC
:1002C000F00AFF001030A0000620F0013030F100ED
:1002D0000830F200F301831203132408F400031022
:1002E000F41B0314F30D0A30F30203187929F30702
:1002F0000310F40DF20B6F29730871070318F00A4D
:10030000FF001030A000062008007F308316031382
:100310009B009F0105088312A5008316060883121F
:10032000A600831605081F3885000608C038860019
:10033000813083129F00A701DC3027020318A22915
:10034000A70A9C291F0804389F001F1DA829A5295A
:1003500025088316850083122608831686009B01D4
:100360000800831203131E0808007F30831603134E
:100370009B009F0105088312A800831606088312BC
:10038000A900831605081F3885000608C0388600B6
:10039000893083129F00AA01DC302A020318D22977
:1003A000AA0ACC291F0804389F001F1DD829D52967
:1003B00028088316850083122908831686009B016E
:1003C0000800831203131E0808007F3083160313EE
:1003D0009B009F0105088312AB0083160608831259
:1003E000AC00831605081F3885000608C038860053
:1003F000993083129F00AD01DC302D020318022AD0
:10040000AD0AFC291F0804389F001F1D082A052A71
:100410002B088316850083122C08831686009B0107
:100420000800831203131E080800DF30F8000000E4
:1004300000000000000000000000000000000000BC
:1004400000000000000000000000000000000000AC
:100450000000000000000000000000000000F80B99
:100460001C2A0000F70B152A000008006430FD006C
:1004700004202030FD0004203D30FD000420203009
:10048000FD0004208316031305160511FB018312DA
:1004900005158312031305081039003C031D5A2A61
:1004A000F0017B08013E0318F00AFB003330F9002D
:1004B0001520492A8312031305117B08A400082084
:1004C000080009200A20FA00142008000B200C2044
:1004D000FA00142008000D200E20FA001420080055
:1004E00064307A0203187E2A2030FD0004200A308E
:1004F0007A0203187E2A2030FD0004207A08831235
:100500000313A400082008000230F90200000000D4
:08051000F90B862A0000080027
:04400E002A3FFC3F0A
:00000001FF
